:100000000C94DB010C94F8010C9413020C94F8018D
:100010000C94F8010C94F8010C94F8010C94F8017C
:100020000C94F8010C94F8010C949D1C0C94F801AC
:100030000C94F8010C94F8010C94F8010C94F8015C
:100040000C94F8010C94F8010C94F8010C94F8014C
:100050000C94F801B105B105DD05DD054506630623
:100060007B077B076E0607071807180700001400B8
:100070001A000800150018000C0012001300E00020
:10008000E30000002B000151000017001C003000AD
:1000900000002F00E10031000000040016000700FE
:1000A00009000D000E000F003300E4002A000000DC
:1000B0000000000000000A000B00000000003400F7
:1000C000E2002C0000001D001B00060019001000BB
:1000D000360037000000E5002800000000000000A6
:1000E000000005001100000076003800E600015114
:1000F0000000165C00000000220023002E0000001B
:100100002D00E700350000001E001F002000210028
:100110002400250026002700000000000000010048
:1001200001000100010001000100010001000100C7
:1001300001000000010001510100010001004D001B
:1001400000004A0001000100000001000100010060
:100150000100510052004F00010001004C0000005E
:10016000000000000000010050000000000001003D
:100170000100010000000100010001000100010078
:100180004B004E00000001000100000000000000D4
:100190000000010001000000010001000100025107
:1001A00000003500000000003E003F004500000058
:1001B00044000100010000003A003B003C003D000B
:1001C0004000410042004300000000000000010028
:1001D0000100010001000100010001000100010017
:1001E00001000000010001510100010001000100B7
:1001F00000000100010001000000010001000100F9
:1002000001000100010001000100010001000000E7
:1002100000000000000001000100000000000100DB
:1002200001000100000001000100010001000100C7
:1002300001000100000001000100000000000000BA
:1002400000000100010000000100010001000100A8
:10025000000001000000000001000100010000009A
:1002600001000100005C000001000100010001002C
:1002700001000100010001000000000009023B0034
:10028000020100A0FA090400000103010100092194
:100290000101000122400007058103080001090453
:1002A00001000103000000092101010001227B007F
:1002B000070583030800011201100100000008A0D7
:1002C000202D420002010200010E0342002E0066B2
:1002D0000061006B00650000001C034E006F00749D
:1002E00000570069006E006B00650079006C0065C6
:1002F000007300730000000403090405010902A152
:100300000185020901A10005091901290815002527
:100310000195087501810205010930093115812512
:100320007F95027508810609381581257F9501752D
:10033000088106050C0A38021581257F950175088C
:100340008106C0C005010980A101850319012AB7F2
:1003500000150126B700950175108100C0050C0934
:1003600001A101850419012AA002150126A0029508
:100370000175108100C005010906A101050719E0FA
:1003800029E7150025019508750181029501750879
:1003900081030507190029FF150026FF0095067542
:1003A0000881000508190129059505750191029537
:1003B0000175039103C011241FBECFE5D8E0DEBF55
:1003C000CDBF10E0A0E6B0E0E8E5F1E402C00590A2
:1003D0000D92A03FB107D9F722E0A0EFB0E001C035
:1003E0001D92A53CB207E1F70E9483130C94AA204A
:1003F0000C940000A82FB92F80E090E041E050EA73
:10040000609530E009C02D9182279795879510F06F
:1004100084279527305EC8F36F5FA8F30895EADF5D
:100420008D939D930895CF93CFB7CF93C395839B1F
:10043000E9F7839B0EC0839B0CC0839B0AC0839B00
:1004400008C0839B06C0C0919C02C395C0939C02C8
:10045000A6C0DF93C0919B02DD27CD55DD4F839B66
:1004600002C0DF91E6CF2F930F931F9300B32FEFBE
:1004700003FB20F94F933F9310B34FEF012703FB8A
:1004800021F93BE031C04E7F012F10B3216028C01D
:10049000102F4D7F2260000000B329C04B7F2460E5
:1004A000012F000010B32BC010B3477F28602AC073
:1004B0004F7E00B320612CC04F7D10B320622FC04F
:1004C0004F7B00B3206432C0422700B349934FEF03
:1004D0000000102713FB20F910B31C70C9F1297F0D
:1004E00091F2012703FB21F900B3237F89F23150F8
:1004F00058F1102713FB22F910B3277E79F2012758
:1005000003FB23F92F7C81F200B3102713FB24F99E
:100510002F7971F200C010B3012703FB25F92F7367
:1005200059F200C000B3102713FB26F9223040F225
:1005300000C010B3012703FB27F9243028F64F77BA
:10054000206810B30000F9CF10E81ABF00271CC0C4
:100550003B503195C31BD04010E81ABF0881033CC3
:1005600011F10B3401F1209198021981110F12132E
:10057000EDCF4A81441F093669F10D3211F0013E79
:1005800029F74F7009F0042F0093A1023F914F917A
:100590001F910F912F91DF91CAB7C7FD47CFCF9120
:1005A000CFBFCF9118952091A102222379F310910A
:1005B0009F02112309F044C034300AF443C0309341
:1005C0009F0220939A0210919B023BE0311B3093D3
:1005D0009B0238C000919F02013094F50AE54F70EC
:1005E00049F43091790034FD2FC000937900C5E7BC
:1005F000D2E02EC0433059F0443091F03091800267
:1006000034FD22C000938002C1E8D2E021C03091C5
:10061000B90234FD19C00093B902CAEBD2E018C088
:1006200030918C0234FD10C000938C02CDE8D2E0F2
:100630000FC02795A8F45150A9F4220F0000F9CF5C
:100640004AE503C042ED01C0432FC4E1D0E032E0EF
:1006500011B31C60939A11BB02B320E41CE05F93BA
:10066000012756E002BB279520F4515021F4220FB8
:10067000F9CF012756E000003B5A02BBD0F2279584
:1006800028F4515029F4220F0000F9CF012756E039
:10069000279502BB20F4515021F4220FF9CF0127F6
:1006A00056E02991332302BB21F6037F1091A0026B
:1006B000110FC651D04002BB11F01093980210E800
:1006C0001ABF086011B3137F402F437F5F9100C0B2
:1006D00000C002BB11BB42BB59CF81E0089581E04D
:1006E00008950C946F0308950C9473031F93CF9394
:1006F000DF9300D000D01F92CDB7DEB749835A8375
:100700006B833091F30089819A81311114C0662383
:1007100059F0222349F00E94B809182F682F8981C7
:100720009A810E94610903C00E948C09182F698177
:100730007A81812F04C00E94B80969817A810F9063
:100740000F900F900F900F90DF91CF911F910C940D
:10075000F410FC01262F40815181628173818481D4
:100760000C94760381E00895CF93DF93EC0160E071
:100770000E94A903BE01DF91CF910C9474030C94E5
:100780003A120C94361208950E940B080E94C3037B
:100790002FEB87E299E0215080409040E1F700C0C4
:1007A00000000C94C31C0F931F93CF93DF938C0115
:1007B00061E00E94A903EC01B8010E947103882343
:1007C00009F444C0B801CE010E9406178823F1F154
:1007D000B801CE010E944A1B8823C1F1B801CE01A5
:1007E0000E94E717882391F1B801CE010E94A61A52
:1007F000882361F1F8018281882309F1CB358DE5E9
:10080000D807C1F050F4C115FCE5DF0781F0CF3DFA
:10081000DC45A9F40E94EF0E19C0CC35EDE5DE07EA
:1008200061F0CD35DD4559F40E94320E08C00E94BA
:10083000C4030CC00E943B0E02C00E943E0EC801C1
:10084000DF91CF911F910F910C946D0380E0DF91A8
:10085000CF911F910F9108950E94471C80E00E9444
:100860003B170C9457040E942A160E945A040C94B9
:100870004D1C08950C94390481E00895CF93C82F3E
:100880000E943C04882329F0C1FF02C0919A01C054
:100890009198CF910895899A91980895CF93C82FF0
:1008A0000E943A048C2F0E943E04CF91089580E06C
:1008B0000C944E040E94A61B0C944E040E94A61B8E
:1008C0009091F200891721F08093F2000C944E046D
:1008D0000895CF93DF93CDB7DEB72B970FB6F8947B
:1008E000DEBF0FBECDBF4F83588769877A878B875E
:1008F00061110E947E0D9E012F5F3F4F86E0F9013E
:1009000011928A95E9F785E0FE013796D9010190A9
:100910000D928A95E1F789819A814C815D81452B01
:1009200031F09F3F31F491E08F3F19F403C091E023
:1009300001C090E090FF09C049815A816B817C81A0
:100940008D819E810E949F0C05C0C9010E94B20347
:100950008111F2CF2B960FB6F894DEBF0FBECDBF3C
:10096000DF91CF910895FC01808191810E94FA0965
:100970000895CF93882309F455C0C82F8CEF8C0FAE
:10098000813AF8F48C2F0E945D1A81114BC06C2FB4
:1009900080916200909163000E94031C882349F0BB
:1009A0006C2F80916200909163000E943B1C0E941A
:1009B000A00D6C2F80916200909163000E94391C01
:1009C0000CC080E28C0F883058F4C77081E001C001
:1009D000880FCA95EAF70E94610DCF910C94A00D83
:1009E000EBE5EC0FE33040F4F0E0E855FF4F808199
:1009F00090E0CF910C94CB1BE8E5EC0FE73150F47D
:100A0000F0E0EE0FFF1FE658FF4F80819181CF91FC
:100A10000C94E11BCD3E30F08C2F0E940814CF9136
:100A20000C94DA14CF910895882389F19CEF980FE4
:100A3000913A40F4682F80916200909163000E9487
:100A40003B1C0DC090E2980F983058F4877091E0ED
:100A500001C0990F8A95EAF7892F0E94670D0C94BF
:100A6000A00D9BE5980F933020F480E090E00C946B
:100A7000CB1B98E5980F973120F480E090E00C9420
:100A8000E11B8D3E20F00E9463140C94DA1408954B
:100A90001F93CF93DF93182FEB010E94B904209787
:100AA00041F087EB9BE00197F1F700C00000219730
:100AB000F6CF812FDF91CF911F910C9414058933CC
:100AC00019F060E070E002C060E570E00C94480549
:100AD000882321F00E94610D0C94A00D08958823B5
:100AE00021F00E94670D0C94A00D0895CF92DF9223
:100AF000EF92FF920F931F93CF93DF937C01D62F3A
:100B0000C72FFC011281058102950F700E94570DBD
:100B10008823B9F01123A9F08C2F807F803421F035
:100B200080E28D0F883068F080914F0282FD09C00D
:100B300082E00E94000E0E94570D91E0D82ED92627
:100B400001C0D12CCC2EC2948FE0C8228C2D90E015
:100B50008C30910508F0CFC1FC01E65DFF4F0C948D
:100B60002F208C2F807FCF70882311F0C295C07FFB
:100B7000112399F0CC2309F4AAC180E28D0F8830AB
:100B800010F0D11104C08C2F0E94610D03C08C2F76
:100B90000E94710D0E94A00D9AC18D2F0E94140514
:100BA000CC2309F4A8C180E28D0F883038F1DD2311
:100BB00029F18C2F0E94770D24C08C2F807FCF705D
:100BC000803211F0C295C07FDD2319F0D130A1F140
:100BD0003DC080914F0282FF17C0112349F0CC2302
:100BE00029F08C2F0E94610D0E94A00D80E070C141
:100BF00080E00E941405CC2309F47DC18C2F0E9453
:100C0000670D0E94A00D77C1112371F0002341F000
:100C1000013031F40E94810D8C2B0E94890D6BC133
:100C20000E94810D8C2B1DC0002319F0013009F4A6
:100C300062C10E94960D25C0112321F0063008F0F4
:100C40005AC10EC0053008F056C11BC0112361F017
:100C5000002331F0F701858180FF39C18F708583D2
:100C60008C2F0E94680547C1002359F0D93309F041
:100C70003FC1FFEF0DEE12E0F15000401040E1F7F0
:100C800035C18C2F0E946F0536C18C2F86958695B5
:100C9000837019F0813061F02EC1112321F08D2F66
:100CA0009C2F937002C080E090E00E94CB1B2BC170
:100CB000112321F08D2F9C2F937002C080E090E0D3
:100CC0000E94E11B20C18D2F112319F00E940814EE
:100CD00002C00E9463140E94DA1415C18C2F837025
:100CE00009F047C011110BC12D2F229526952770B1
:100CF000220F220F6D2F6F70862F90E0A0E0B0E0E2
:100D0000022E04C0880F991FAA1FBB1F0A94D2F796
:100D1000D4FF10C04FE050E060E070E004C0440F2A
:100D2000551F661F771F2A95D2F7409550956095FD
:100D3000709503C040E050E0BA01C695C695C370F7
:100D40008A019B01082B192B2A2B3B2BC901B801C7
:100D5000C23049F058F4C13019F00E947708CFC072
:100D60000E946508CCC00E948908C9C00E9463081F
:100D7000C6C0112319F08C2F817001C0869588237D
:100D800009F4BDC02D2F229526952770220F220F22
:100D90006D2F6F70862F90E0A0E0B0E0022E04C0AF
:100DA000880F991FAA1FBB1F0A94D2F7D4FF10C047
:100DB0004FE050E060E070E004C0440F551F661F34
:100DC000771F2A95D2F7409550956095709503C08E
:100DD00040E050E0BA01C695C695C3708A019B01F8
:100DE000082B192B2A2B3B2BC901B801C23049F023
:100DF00058F4C13019F00E943C0981C00E942A09B0
:100E00007EC00E944E097BC00E949D0878C0CF70B2
:100E1000112339F08C2F0E94C3088D2F0E94680582
:100E20006EC08D2F0E946F058C2F0E94E40867C052
:100E3000D23F21F128F4D03F41F0D13FC1F043C06F
:100E4000D33F19F1D43F79F03EC0112341F0053072
:100E500008F051C08C2F8F710E9409094CC00630D8
:100E600008F049C0F7CF80914F0282FF18C01123CC
:100E700039F08C2F8F710E94C3083DC01123C9F334
:100E80008C2F8F710E94E40836C0112329F08C2F1B
:100E90008F710E94AE082FC00E94A9082CC0112398
:100EA00049F0CF718C2F0E94C30863E08C2F0E9401
:100EB000E50D21C081E00E94000E0230E0F082E0EA
:100EC0000E94000E18C0112331F0002391F28D2FE3
:100ED0000E94B90410C0002399F2D93349F41FEFDE
:100EE0002DEE32E0115020403040E1F700C000000C
:100EF0008D2F0E94140588EF8C0D843020F40E9401
:100F0000A61B0E944E04DD20C9F00E94530D80FDF7
:100F100015C0F70112820E944D0D0E94C308C7013F
:100F20000E94BF070E944D0DDF91CF911F910F913D
:100F3000FF90EF90DF90CF900C94E408DF91CF9179
:100F40001F910F91FF90EF90DF90CF9008950F9336
:100F50001F93CF93DF93EC01688179818A810E948E
:100F6000050A8C010E9460090E945108B801CE0157
:100F70000E947605DF91CF911F910F910895CF9335
:100F8000DF93EC01988189812B813C81232B31F007
:100F90008F3F31F481E09F3F19F403C081E001C02D
:100FA00080E080FD1DC0CE010E94D303811110C0DE
:100FB0000E94570D8823A1F08A81882389F08091AF
:100FC0004F0282FD0DC082E0DF91CF910C94000EA4
:100FD000CE010E94A707CE01DF91CF910C94B403FC
:100FE000DF91CF91089580E090E00E94CB1B80E0DC
:100FF00090E00E94E11B0E947E0D0E94A00D0E94C5
:101000000B160C94DA1480916200909163000E9498
:101010003D1C0C94F3070E946E0D0C9403089295EE
:101020009F70963079F010F4925001C09A5092302F
:1010300068F4803F69F018F4883E40F409C0843FAA
:1010400029F406C0883E20F0813F11F080E0089529
:1010500081E00895FC01808191810E94FA090E943B
:101060000F080895CF93DF9300D000D01F92CDB723
:10107000DEB70F900F900F900F900F90DF91CF91F0
:101080000895CF93DF9300D000D000D0CDB7DEB766
:1010900026960FB6F894DEBF0FBECDBFDF91CF917D
:1010A0000895089508950C9452080C9453080E94D2
:1010B000550860932F017093300180933101909314
:1010C00032010C94F3070C9457080F931F9300916F
:1010D0002F01109130012091310130913201602BAC
:1010E000712B822B932B1F910F910C9457080F9308
:1010F0001F9300912F011091300120913101309107
:10110000320160237123822393231F910F910C944A
:1011100057080F931F9300912F01109130012091D8
:1011200031013091320160277127822793271F9167
:101130000F910C9457080C9452080E949B086093DE
:101140002B0170932C0180932D0190932E010C9410
:10115000F30760E070E0CB010C949D080F931F93A0
:1011600041E050E060E070E08A019B0104C0000FA4
:10117000111F221F331F8A95D2F7C901B8011F9191
:101180000F910C949D080F931F9341E050E060E095
:1011900070E004C0440F551F661F771F8A95D2F771
:1011A00080912B0190912C01A0912D01B0912E01E5
:1011B0008A019B01082B192B2A2B3B2BC901B80153
:1011C0001F910F910C949D080F931F9341E050E0E5
:1011D00060E070E004C0440F551F661F771F8A95BA
:1011E000D2F7409550956095709580912B01909124
:1011F0002C01A0912D01B0912E018A019B010823A1
:1012000019232A233B23C901B8011F910F910C9484
:101210009D080F931F9341E050E060E070E004C030
:10122000440F551F661F771F8A95D2F780912B01B7
:1012300090912C01A0912D01B0912E018A019B016A
:10124000082719272A273B27C901B8011F910F91A9
:101250000C949D080F931F9300912B0110912C016A
:1012600020912D0130912E01602B712B822B932B1D
:101270001F910F910C949D080F931F9300912B01C8
:1012800010912C0120912D0130912E0160237123AA
:10129000822393231F910F910C949D080F931F930A
:1012A00000912B0110912C0120912D0130912E01E4
:1012B00060277127822793271F910F910C949D0817
:1012C00008952BE0929F800D1124E82FE695E69576
:1012D000E695877051E001C0550F8A95EAF785E0E1
:1012E000E89FF0011124EC50FF4F20E030E070E067
:1012F0004081CB01022E02C0969587950A94E2F7B1
:101300008170819584278523842781932F5F3F4FA8
:101310002530310569F708952BE0929F800D112447
:10132000682F669566956695982F977085E0689FFB
:10133000B001112440E050E080E0FB01E40FF51F14
:10134000EC50FF4F208130E0092E02C036952795E2
:101350000A94E2F721703327042E01C0220F0A9469
:10136000EAF7822B4F5F5F4F4530510531F7089503
:10137000BF92CF92DF92EF92FF920F931F93CF9382
:10138000DF938C01C0902B01D0902C01E0902D01B7
:10139000F0902E0180912F0190913001A0913101A8
:1013A000B0913201C82AD92AEA2AFB2ACFE1D0E03B
:1013B000D701C6010C2E04C0B695A79597958795C1
:1013C0000A94D2F780FD04C0219790F7B12C07C092
:1013D000BC2EB8018C2F0E9407110197A9F38B2D09
:1013E000DF91CF911F910F91FF90EF90DF90CF9001
:1013F000BF900895CF93DF93EC010E94B809BE011E
:101400000E940711DF91CF9108951F93CF93DF932F
:10141000EB019091F300992321F0CB010E94FA098E
:1014200013C0882349F0CB010E94B809182F682FF8
:10143000CE010E94610904C0CB010E948C09182FC3
:10144000BE01812F0E940711DF91CF911F91089556
:101450001F93CF93DF93C091330116E08091340145
:10146000C81799F0D0E01C9FF0011D9FF00D1124CA
:10147000EB5CFE4F40815181628173818481958153
:101480000E9441082196C770E9CFDF91CF911F914B
:1014900008954091650150916601609167017091D6
:1014A00068018091690190916A010C944108EF9262
:1014B000FF920F931F93CF93DF9380916A018295E0
:1014C0008F7009F065C080916701882309F460C0BE
:1014D00080913301F0903401109165010091660113
:1014E000609168017091690191E01F3F09F090E0FF
:1014F000C0916000D0916100292F96E0E92E8F15F0
:1015000009F446C06115710521F00F3F21F030E06C
:1015100003C031E001C0322F90E030FD36C0E89EBC
:10152000F001E99EF00D1124DF01AB5CBE4F119676
:101530003C911197301329C03C91311326C012966B
:101540003C911297311121C013964D915C911497E3
:10155000461B570B4C175D07C0F480916A018F70D2
:10156000806180936A01E65CFE4F80818F708061AC
:10157000808385E691E00E94BF07DF91CF911F91A4
:101580000F91FF90EF900C94280A01968770B7CFC7
:10159000DF91CF911F910F91FF90EF9008959F924F
:1015A000AF92BF92CF92DF92EF92FF920F931F9371
:1015B000CF93DF93CDB7DEB761970FB6F894DEBF58
:1015C0000FBECDBF8C0185E0F801DE011D960190B4
:1015D0000D928A95E1F7D8011296EC9090916501F1
:1015E000E091660120916801309169012115310572
:1015F00031F0EF3F31F481E09F3F19F403C081E007
:1016000001C080E0B82FB1709B2E80FD47C1D8018A
:101610004C9111965C9111971396AD90BC901497D4
:1016200085E6C82E81E0D82EF0906701B501621BD7
:10163000730B2091600030916100FF2009F4D9C044
:1016400080916A016217730708F095C0282F207FE8
:1016500009F052C05E1313C0491311C0FE2CE110F3
:101660000EC08F70806180936A010E94490AC60192
:101670000E94BF0780916A01F80185834DC1AB28A4
:1016800031F05F3F31F481E04F3F19F403C081E056
:1016900001C080E080FD03C081E08E2502C080E0B3
:1016A00090E0F82FF170FF2E80FF1CC08091330175
:1016B0002091340136E0821709F40BC190E0389F85
:1016C000F001399FF00D1124EB5CFE4F6181561340
:1016D00006C06081461303C06281E61203C0019612
:1016E0008770E9CFFE2CEE2009F416C180916A01C3
:1016F000816080936A0154C05E1306C0491304C020
:10170000E11002C0F80199C0C8010E942A0888238C
:1017100061F1EE2051F120916A01822F82958F7044
:1017200090E0029774F0809165019091660198872E
:101730008F831986BB86AA862C87CE0107960E94C6
:10174000BF0786E0F801A5E6B1E001900D928A9509
:10175000E1F70E94570A0E94490A0AC05E1711F178
:10176000C8010E942A0881112CC0C8010E94BF072D
:10177000FF24F394D1C0282F207F81F77A2DB98AD6
:10178000A88A6E2D89890E94320885E691E00E9420
:10179000BF0786E0D6011D928A95E9F70E94490AA3
:1017A000F12CBAC04913DCCFE110DACFF801858300
:1017B000C8010E94BF0786E0D6011D928A95E9F70D
:1017C000ABC0EE2091F220916A01822F82958F703A
:1017D00090E002970CF4B5CF80916501909166017D
:1017E0009A8389831B82BD82AC822E83CE010196AF
:1017F000A6CF6217730708F044C0FE2CEE2009F450
:10180000B4CF5E1330C049132EC020916A0120FD71
:1018100021C0822F82958F70482F50E041155105CD
:10182000C9F0F80125834F30510541F08F5F982FA3
:101830009295907F822F8F70892B8583C8010E949B
:10184000BF0786E0F801A5E6B1E001900D928A9508
:10185000E1F73CC086E0F801A5E6B1E001900D9209
:101860008A95E1F759C0C8010E942A08811169CF01
:1018700080916A01816080936A01C8010E94BF075C
:101880004BC07A2DB98AA88A6E2D89890E943208A8
:1018900086E0D6011D928A95E9F718C0EE2009F47A
:1018A00064CFC8010E942A08F82E882309F45DCF6E
:1018B00086E0F801A5E6B1E001900D928A95E1F786
:1018C00085E691E00E94B3040E94570A0E94490AEB
:1018D00023C04D875E878D859E850E94FA09292F3A
:1018E00022952F70223028F49F7039F0811105C0A5
:1018F0000BC0243028F49F7049F4805E883020F0BB
:10190000C8010E94BF079F2CF92C06C0D80115966C
:101910009C91907F91F7F8CF8F2D61960FB6F89438
:10192000DEBF0FBECDBFDF91CF911F910F91FF9012
:10193000EF90DF90CF90BF90AF909F9008951F934E
:10194000CF93DF93CDB7DEB72C970FB6F894DEBFF9
:101950000FBECDBF4F83588769877A878B879C8757
:10196000CE0107960E94CF0A8823D1F09F818885F7
:101970002A853B85232B31F08F3F31F481E09F3F57
:1019800019F403C081E001C080E080FD47C04F81B1
:10199000588569857A858B859C850E9441083EC063
:1019A00086E0FE013796DE01119601900D928A9530
:1019B000E1F7FF81E8856A857B856115710531F066
:1019C000EF3F31F481E0FF3F19F403C081E001C033
:1019D00080E080FD23C02091340130E0C9010196F0
:1019E000877099274091330150E084179507F1F1F2
:1019F000F983EA837D836C8396E0929FD001939F65
:101A0000B00D1124AB5CBE4FFE01319601900D92DA
:101A10009A95E1F7809334010E94280A16E080919C
:101A2000330190913401891771F1189FC00111247D
:101A30008B5C9E4F0E94CF0A882329F1E0913301ED
:101A40001E9FF0011124EB5CFE4F408151816281A9
:101A50007381848195810E9441088091330190E0D7
:101A600001968770992780933301D9CF0E940B0884
:101A70001092340110923301E5E6F1E086E0DF01D7
:101A80001D928A95E9F72C960FB6F894DEBF0FBE2B
:101A9000CDBFDF91CF911F910895809173018595FE
:101AA000859585950895809173018770089590912B
:101AB0007301977081E009F480E0089580917E01C0
:101AC000089590917E01892B80937E0108958095E1
:101AD00090917E01892380937E01089510927E016A
:101AE000089590917D01892B80937D0108958095C3
:101AF00090917D01892380937D01089510927D014D
:101B0000089580917401089508950C94840D0C94A7
:101B1000850D90914F0292FD08C090917401981725
:101B200021F0809374010C94870D089580917401C5
:101B3000882329F01092740180E00C94870D089599
:101B4000CF93DF93E0916200F091630080917E017A
:101B50008083E0916200F0916300908180917D012B
:101B6000892B808380917401882381F0E091620049
:101B7000F09163009081892B808380916200909125
:101B800063000E94F71B81110E94960DC0916200B4
:101B9000D091630048E050E06BE671E0CE010E9416
:101BA0004F20892B69F088E0FE01ABE6B1E001909F
:101BB0000D928A95E1F7CE01DF91CF910C94B21B83
:101BC000DF91CF9108950C94840D90914F0292FD76
:101BD00010C098E0899F90011124262B2093730157
:101BE0000E94C308809173018595859585950C9415
:101BF000E30D0C94C3081092730180E00C94E30D84
:101C0000209173018095822380937301982F9770A0
:101C100099F430E0482F082E000C550B2417350797
:101C200059F090914F0292FD07C085958595859555
:101C30000E94E4080C94FB0D089590914F0292FBD2
:101C4000222720F9281769F080FB92F990934F0220
:101C500080914E0290914F020E946B0E82E00C9494
:101C6000000E089580914F0282FB882780F991E051
:101C700089270C941D0E81E00C941D0E80E00C94BD
:101C80001D0E6FEF7FEF80E090E00C94872080E0E6
:101C900090E00E94642021E0893E9E4F09F020E000
:101CA000822F089582E090E00C945C2083E090E025
:101CB0000C945C20CF9384E090E00E945C20C82FBD
:101CC00082E290E00E945C202C2F30E0A901582B8A
:101CD000CA01CF910895CF93C92F682F84E090E077
:101CE0000E946A206C2F82E290E0CF910C946A20CF
:101CF000AB01BC018FE090E00C947B20AB01BC01F8
:101D000083E190E00C947B2060E070E0CB010C94C8
:101D10007E0E60E070E0CB010E94780E0C94840E81
:101D200069EE7EEF80E090E00E94872060E082E034
:101D300090E00E946A2060E083E090E00E946A20C8
:101D400010922F0110923001109231011092320145
:101D500060E084E090E00E946A2060E082E290E02F
:101D60000E946A2060E085E090E00E946A2060E0C6
:101D700086E090E00E946A206FEF87E090E00E948A
:101D80006A2040E050E0BA0188E090E00E947B20A9
:101D900060E08DE090E00E946A2040E050E0BA01EF
:101DA00088E190E00E947B2060E087E190E00E9463
:101DB0006A2040E050E0BA018CE190E00E947B2074
:101DC00060E070E080E290E00E94872040E050E018
:101DD000BA0188E190E00E947B200C94890E0C945B
:101DE000900E682F8EE090E00C946A200E94821C76
:101DF0006093930170939401809395019093960161
:101E000060938F0170939001809391019093920160
:101E1000089584B7806884BF84B7806884BF0895BC
:101E200081E008950C94100F08950C94140F0C94F5
:101E3000140F0C94170F0C94140F0C941B0F0C948C
:101E4000140F0E94090F83EE91E10E949C1B0E94D7
:101E50001F0F0C941D0F0E94150F0C94140F0E945D
:101E6000FD110E944B040C94DB170E946F1C0E9412
:101E7000E2120E942F0F0E942A160C94190F5F92F3
:101E80006F927F928F929F92AF92BF92CF92DF928A
:101E9000EF92FF920F931F93CF93DF93CDB7DEB7EF
:101EA0002A970FB6F894DEBF0FBECDBF0E94F7127F
:101EB000C82E81110E94F60E3FE7832E31E0932E4B
:101EC00000E010E0502E802F0E9421125C01F401EE
:101ED000619071904F016826792661147104B1F404
:101EE0000F5F1F4F0830110569F78FEF89838A83D1
:101EF0001B820E94761C8160782F9D838C83498190
:101F00005A816B818D810E9469043AC0809197014A
:101F100081FD0E942A12D12CEE24E394F12CC301FE
:101F20008E219F21892B29F10E94120F8823A9F06D
:101F3000DE825F82AE20BF2081E0AB2809F480E022
:101F400088870E94761C8160782F9A8789874E81C6
:101F50005F8168858A850E946904000F111FF8015E
:101F6000E158FE4F80819181E826F926F182E082D6
:101F700007C0D394EE0CFF1CFBE0DF12D0CFB0CF34
:101F800081E0C11001C080E02A960FB6F894DEBF50
:101F90000FBECDBFDF91CF911F910F91FF90EF90BA
:101FA000DF90CF90BF90AF909F908F907F906F9079
:101FB0005F9008950E943F0F0E94DA170E94F81464
:101FC0000C945E04CF93DF930E940C11EC018115F9
:101FD00021E5920708F045C0811530E5930708F028
:101FE00094C0883E910528F5803E910508F0F8C020
:101FF000883A910570F4853A910508F07CC08130EB
:10200000910509F475C008F4E8C0049708F0E8C029
:10201000E4C08F3B910508F0E0C0C85AD0E0CC0F77
:10202000DD1FC555DF4F0990D881C02DCE019464C6
:10203000D8C0811540E2940758F4811551E0950706
:1020400008F0CEC08D3E910508F4C7C09065C9C0A8
:10205000C11580E4D80708F4C0C0DF70CE01906AD3
:10206000C0C0811525E59207A8F4811534E59307D2
:1020700008F095C0811543E5940708F07BC08115F1
:1020800052E5950708F061C0D82FCC27CE01816FAB
:10209000906AA7C0C11589E5D807A0F4C11528E545
:1020A000D20708F082C0C11536E5D30708F095C005
:1020B0008C2F0E94A0118F7190E0D82FCC27CE01D9
:1020C00090628FC0C1154AE5D40708F474C0CE01F0
:1020D00090568115904208F080C08D2F8F710E941C
:1020E000A011DD27D0628F71AE01582BCA0179C0D3
:1020F00081E090E076C0C55AD0E0C752DF4F8881BA
:10210000C82FD0E0CE0190646CC074E0969587959E
:102110007A95E1F7282F23703C2F337081E090E00F
:1021200002C0880F991F3A95E2F79C68AC01522BC8
:102130009A019C2F9F709695969550E2959FE0018D
:102140001124C9018C2B9D2B4CC08370992721E051
:1021500030E002C0220F331F8A95E2F79C2F96953C
:10216000969580E2989FE0011124C22BD32BCE01DB
:102170009C6837C08370992721E030E002C0220FAD
:10218000331F8A95E2F79C2F9695969540E2949F8F
:10219000E0011124C22BD32BCE019A6822C0D82F84
:1021A000CC27CE01846F906A1CC0DC2FCC27CE01D7
:1021B000806F906A16C08C2F8F700E94A01194E0DF
:1021C000D695C7959A95E1F7CF70D0E0DC2FCC2754
:1021D000D0699E01282BC90104C080E090E001C0B5
:1021E000CE01DF91CF91089528E5829FC00111248F
:1021F000FC012BE0729FE00DF11D1124E60FF11D93
:10220000EE0FFF1FE459FF4F8591949108950E94AE
:10221000F4100E94E20F08958238910569F1B0F43C
:102220008133910509F46DC048F48932910509F4B0
:1022300063C08A32910509F469C008958533910518
:1022400009F455C089339105B9F00895833E91058D
:1022500069F138F4803E9105B1F0823E910509F1B3
:102260000895863E9105A9F1873E9105B9F1843E16
:10227000910509F064C023C020914E0220FD4FC09B
:1022800021FD4DC0089580914E0280FD44C0809193
:102290004F0280FF44C080914E0284FD42C083EE15
:1022A0004DC080914E0282FF38C0F5CF80914E0222
:1022B00082FD33C080914F0280FD31C0ECCF809110
:1022C0004F0281FF32C080914E0284FD2AC087EE0A
:1022D00035C080914E0283FF26C0F5CF80914E021B
:1022E00083FD21C080914F0281FD1FC0ECCF809102
:1022F0004E0285FD1CC01DC080914E0285FD19C097
:1023000016C080914E0286FD16C017C080914E0205
:1023100086FD13C010C089E311C082EE0FC080EEAD
:102320000DC080E00BC086EE09C084EE07C089E2D4
:1023300005C085E303C08AE201C081E390E008950F
:1023400090914E0292FF0DC0282F2871283019F469
:10235000877F846006C0282F2471243011F48B7F7E
:10236000886093FF0DC0282F2871283119F4877ECB
:10237000846106C0282F2471243111F48B7E88617A
:1023800020914F0220FF0DC0382F3871383019F4DA
:10239000877F816006C0382F3171313011F48E7F14
:1023A000886021FF0DC0282F2871283119F4877EFD
:1023B000816106C0282F2171213111F48E7E886140
:1023C00094FD877E089580E008950C94410E0E944C
:1023D000F7128FE295E70197F1F700C000000E9425
:1023E000F71280E00E94211280FF04C00E94E511D4
:1023F0000C94C31C08950C94E7110E94470E8111A0
:1024000002C00E94EF0E0E94520E809397010E941C
:102410005A0E90934F0280934E020E94FB110E942D
:10242000560E682F70E080E090E00E946308609193
:102430002B0170912C0180912D0190912E010C9413
:102440009B08E82FF0E0EE0FFF1FE05AFD4F808160
:1024500091810895089588E78A95F1F7089500C05D
:1024600008950C942B1208950C9433120C9434128A
:102470000C9433120C943812F894E82FE295EF7014
:10248000F0E031A9282F2F7081E090E001C0880F83
:102490002A95EAF7982F9095932391AB92A9892BCF
:1024A00082AB789408950F931F93CF93DF93C7EE79
:1024B000D0E089918F3F11F00E943C1280E0CF3E26
:1024C000D807B9F7CCEDD0E007EE10E089918F3F47
:1024D00011F00E943C120C171D07C1F7DF91CF913C
:1024E0001F910F910895BF92CF92DF92EF92FF92CA
:1024F0000F931F93CF93DF938C01C62FD0E0CE01B3
:1025000089519F4F6C01FC0190819F3F09F450C09D
:10251000B62EF894E92FE295EF70F0E081A99F7054
:1025200021E030E001C0220F9A95EAF7822B81ABBF
:1025300082A92095282322AB78940E942F12ECEDDB
:10254000F0E047EE50E021E030E0E12CF12C619129
:102550006F3F89F0A62FA295AF70B0E0D0968C9116
:1025600090E06F7002C0959587956A95E2F780FDBF
:1025700002C0C90102C080E090E0E82AF92A220FD7
:10258000331F4E175F0719F7F60180818F3F11F057
:102590000E943C1261E0E114F10409F460E08B2D2B
:1025A0000E943112CC0FDD1FC00FD11FF982E882CB
:1025B000DF91CF911F910F91FF90EF90DF90CF901F
:1025C000BF9008950E94531280E1E0E6F2E0DF013F
:1025D000982F1D929A95E9F7E0E5F2E0DF011D9250
:1025E0008A95E9F788E00E9442130C94BF03FF929A
:1025F0000F931F93CF93DF93CDB7DEB760970FB6DE
:10260000F894DEBF0FBECDBF8E010F5F1F4F80E17C
:10261000F80111928A95E9F7F12C6F2DC8010E94FB
:102620007312F394F8E0FF12F8CF40E150E0B801E4
:1026300080E592E00E944F20FF24F394009709F474
:10264000F12C892B41F080E1F801A0E5B2E0019086
:102650000D928A95E1F72F2D48E060E672E080E563
:1026600092E00E9443130E94C1038F2D60960FB623
:10267000F894DEBF0FBECDBFDF91CF911F910F91B8
:10268000FF9008950895FF920F931F93CF93DF93C8
:10269000F82E092F162FD72FC42F222349F081E0BF
:1026A00080939A010E94761C9093990180939801DF
:1026B00080919A018823D9F0809198019091990195
:1026C0000E948E1C059798F0EF2DF02FA12FBD2FA3
:1026D00080E090E04C2F50E08417950734F421916E
:1026E00031912D933D930196F7CF10929A01DF918E
:1026F000CF911F910F91FF9008950E94D81C0E94C6
:10270000350F0C94E91C0E94641C0E94D11C0E948D
:10271000210F0E947D130E94F71C0E942B0FFBCFFC
:102720008091A10180FF06C06091690070E0660F92
:10273000771F26C081FF04C06091690084E005C056
:1027400082FF07C06091690088E0689FB001112492
:1027500017C09091A0019923D1F06091680096175D
:1027600088F72091690088E0289F90011124929FAA
:10277000A001939F500D112470E0CA010E94F91F1F
:102780006038710540F46115710519F406C068E000
:1027900070E0862F08958FE7089581E00895809175
:1027A000A10180FF08C06091650070E07595679594
:1027B0007595679521C081FF06C06091650070E046
:1027C0007595679519C082FF04C06091650070E03F
:1027D00010C090919F01992399F060916400961721
:1027E000A0F780916500899FC001112470E00E94CC
:1027F000F91F6038710540F46115710519F406C0C0
:1028000061E070E0862F08958FE7089581E00895D4
:102810008D3E21F40E949013819504C08E3E29F4D0
:102820000E9490138093A50108958F3E21F40E9489
:102830009013819504C0803F29F40E9490138093E7
:10284000A4010895893F19F40E94CF1305C08A3F5F
:1028500031F40E94CF1381958093A60108958B3F98
:1028600021F40E94CF13819504C08C3F29F40E946B
:10287000CF138093A70108959FE0980F983078F4C4
:1028800021E030E0A90102C0440F551F9A95E2F7FC
:10289000CA019091A301892B8093A30108958D3FD4
:1028A00021F48091A10181600BC08E3F21F48091C1
:1028B000A101826005C08F3F29F48091A10184604D
:1028C0008093A10108958D3E39F49091A50197FF61
:1028D00035C01092A50159C08E3E29F49091A501F2
:1028E0001916BCF32BC09091A4018F3E29F497FFD9
:1028F00025C01092A40149C0803F19F41916CCF3E9
:102900001DC09091A601893F29F41916BCF41092BC
:10291000A6013BC08A3F19F497FF10C0F8CF8B3F48
:1029200039F49091A70197FF09C01092A7012DC01B
:102930008C3F21F49091A7011916BCF39FE0980FEA
:10294000983080F421E030E0A90102C0440F551F07
:102950009A95E2F7CA0180959091A301892380930B
:10296000A30113C08D3F21F48091A1018E7F0BC084
:102970008E3F21F48091A1018D7F05C08F3F29F406
:102980008091A1018B7F8093A1018091A40181118D
:1029900006C08091A501811102C01092A001809112
:1029A000A601811106C08091A701811102C0109279
:1029B0009F0108950E94761C2091A401211104C05A
:1029C0002091A501222321F090939E0180939D01E7
:1029D0002091A601211104C02091A701222321F0FA
:1029E00090939C0180939B0182EA91E00C94BD1B23
:1029F000EF92FF920F931F93CF93DF9300D000D0FD
:102A000000D0CDB7DEB786E0E2EAF1E0DE01119654
:102A100001900D928A95E1F7E090A401F090A50154
:102A20000091A6011091A7011092A4011092A50196
:102A30001092A6011092A701E11003C0FF2009F433
:102A40005DC080919D0190919E010E948E1CAC0101
:102A50009091A001992339F020916A0030E0241769
:102A6000350758F04BC020916B008AE0289F9001F9
:102A700011242417350718F041C09F3F19F09F5FBC
:102A80009093A001EE2061F00E9490131E1414F0A8
:102A90009FEF01C091E0989F902D11249093A40185
:102AA000FF2061F00E9490131F1414F09FEF01C0EB
:102AB00091E0989F902D11249093A5013091A4014D
:102AC0003323E1F02091A5012223C1F045EB34032B
:102AD000C0011124992319F09093A40103C081E04F
:102AE0008093A40135EB2303C0011124992319F02D
:102AF0009093A50103C081E08093A501011103C05B
:102B0000112309F45DC080919B0190919C010E946A
:102B10008E1CAC0190919F01992339F020916600A1
:102B200030E02417350758F04BC0209167008AE049
:102B3000289F900111242417350718F041C09F3FAA
:102B400019F09F5F90939F01002361F00E94CF13C3
:102B5000101614F09FEF01C091E0989F902D112462
:102B60009093A601112361F00E94CF13111614F067
:102B70009FEF01C091E0989F902D11249093A701A1
:102B80003091A6013323E1F02091A7012223C1F067
:102B900045EB3403C0011124992319F09093A60149
:102BA00003C081E08093A60135EB2303C00111240B
:102BB000992319F09093A70103C081E08093A701A6
:102BC0008091A40181110BC08091A501811107C0E2
:102BD0008091A601811103C08091A70181110E94FB
:102BE000DA14EB82FC820D831E8386E0FE013196AF
:102BF000A2EAB1E001900D928A95E1F726960FB610
:102C0000F894DEBF0FBECDBFDF91CF911F910F9122
:102C1000FF90EF900895E2EAF1E086E0DF011D9277
:102C20008A95E9F71092A00110929F011092A101DC
:102C3000089586E090E00C945C20682F86E090E098
:102C40000C946A2080917002847089618093700274
:102C50000C941D160E94470E811104C00E94EF0EB5
:102C60000E9422160E94191680937002282F269522
:102C70002695269530E02430310524F08770886150
:102C8000809370028091700280FF04C086958695C3
:102C9000869501C080E00C943B1720917002822F32
:102CA000869586958695482F50E04330510554F41B
:102CB0008F5F982F990F990F990F822F8770892B0B
:102CC00080937002809170028160809370020E94F4
:102CD0001D16809170028695869586950C943B17FB
:102CE00080917002982F969596959695A1F0915E99
:102CF000990F990F990F8770892B80937002887FA5
:102D000091E009F490E08091700290FB80F980934B
:102D100070020E941D168091700286958695869598
:102D20000C943B178091700280FD13C081608093EA
:102D30007002813019F489E08093700280917002F2
:102D40000E941D16809170028695869586950C943A
:102D50003B1708958091700280FF08C08E7F80939A
:102D600070020E941D1680E00C943B17089580911C
:102D7000700280FD0C94AA160C9492169091700229
:102D8000892F8695869586958F5F8F719770843091
:102D900038F4880F880F880F892B8093700202C047
:102DA0009093700280917002887F91E009F490E026
:102DB0008091700290FB80F9809370020E941D1632
:102DC000809170028695869586950C943B17843089
:102DD00008F083E0909170029770282F220F220F45
:102DE000220F922B90937002987F21E009F420E04B
:102DF0009091700220FB90F9909370020C943B1715
:102E00000E94E716809170020C941D169C01FB0134
:102E10008281882349F12E3BFCE53F07C9F040F44D
:102E20002C3BECE53E0769F02D3B3C4561F00895F5
:102E3000203C9CE5390791F070F0213C3C4589F03D
:102E4000089583E001C080E00E94001780E00895AB
:102E50000E947016FBCF0E944D16F8CF0E94B71645
:102E6000F5CF0E94BE16F2CF81E008958C9A949817
:102E70000895949808958F929F92AF92BF92CF92A7
:102E8000DF92EF92FF920F931F93CF93DF93C82FA0
:102E9000843040F4811107C08FB58F7D8FBD0E94B3
:102EA000391704C0C3E08FB580628FBDA6B5B7B532
:102EB0002C2F30E00E94352023E030E040E050E04D
:102EC0000E940D200027122F232F342F012F122FA5
:102ED000232F332786B597B56CE070E00E94E51F7D
:102EE0006017710730F0C80169E070E00E94E51FCB
:102EF00052C086B597B5E6B4F7B4E6B5F7B5C6E007
:102F0000D0E0BE010E94E51F060F171F211D311DD5
:102F10004801590185E0880C991CAA1CBB1C8A95A4
:102F2000D1F7C701BE010E94E51F6F01E12CF12C12
:102F3000A7019601260F371F411D511DC501B40180
:102F40000E940D2069017A01E6B5F7B5CA01B90101
:102F50000E94D51F9B01AC01DF010E9444209B0110
:102F6000AC01C701B6010E94D51FDC01CB012FE0E7
:102F7000B695A795979587952A95D1F706B517B574
:102F800020E030E0081719072A073B0718F466B558
:102F900077B5CB01BC0179BD68BDDF91CF911F91A1
:102FA0000F91FF90EF90DF90CF90BF90AF909F90E8
:102FB0008F90089508950E94361782E28FBD89E1AF
:102FC0008EBD8FEF9FEF97BD86BD0C942A16CF93D1
:102FD000DF93EC01FB018281882309F43CC1C430FA
:102FE000FDE5DF0760F4CB3F9CE5D90788F49E013F
:102FF00022503C452431310508F02EC109C0C236AB
:10300000EDE5DE0729F0C63AFDE5DF0709F024C14A
:103010000E945A0E90934F0280934E02C1318CE56C
:10302000D80709F4C6C008F042C0C930ECE5DE0795
:1030300009F49BC000F5C5308CE5D80709F485C0BC
:1030400078F4C330ECE5DE0709F478C008F07AC004
:10305000C230DC4509F0F5C080914E028160EFC0BE
:10306000C7309CE5D90709F478C008F07AC0809190
:103070004E028061E4C0CD30FCE5DF0709F487C073
:1030800058F4CB309CE5D90709F479C008F07BC02F
:1030900080914E0288606FC0CF30FCE5DF0709F4F5
:1030A00080C008F082C080914E02877FC8C0CE3FAA
:1030B0009CE5D90709F471C000F5C531FCE5DF07CF
:1030C00009F485C068F4C3319CE5D90709F475C0DB
:1030D00008F095C00E940B0880914E028F77AFC018
:1030E000CC3FFCE5DF07A9F108F054C0CB3FDC453D
:1030F00009F0A7C080914F0240C0C230EDE5DE0765
:1031000009F489C058F4C1158DE5D80709F45AC0EF
:1031100008F069C080914F0282602FC0C236EDE591
:10312000DE0709F47CC0C63AFDE5DF0709F481C07B
:10313000C330DD4509F085C080E06EC080914E024D
:1031400082607DC080914E0216C080914E028860E0
:1031500076C080914F0282604FC080914E028062A3
:103160006EC080914E0280646AC00E940B088091FC
:103170004E02806864C0846062C081603DC08091FE
:103180004E028E7F5CC080914E028D7F58C0809130
:103190004E0216C080914F0218C080914F028D7F61
:1031A0002BC080914E028F7E4AC080914E028F7D4F
:1031B00046C080914E028F7B42C080914E02877F35
:1031C0008B7F3DC080914F028D7F8E7F15C0809197
:1031D0004E0282FB222720F991E0922790FB82F990
:1031E00090FB83F92CC080914F02982F909591709D
:1031F0008E7F892B90FB81F980934F0222C00E9421
:103200000B0880914E0287FB222720F991E092273C
:1032100090FB87F914C081E00E94F10E12C08091EA
:103220004E0284FB222720F991E0922790FB84F93B
:1032300006C080914E02982F909590FB80F9809364
:103240004E0280914E0290914F020E946B0E0E949E
:103250000B0880E001C081E0DF91CF9108958932B1
:1032600089F1F0F4843171F1B0F4873009F077C05E
:1032700081E080936B0084E180936A008AE0809310
:1032800069008EE18093680088E08093650088E2A1
:103290008093640064C092EE980F9A30F0F05FC0A3
:1032A000803509F444C028F48F3409F058C08AE00E
:1032B0003FC0813529F0823509F051C081E038C026
:1032C0008FEF36C08091AA01882379F11092AA016C
:1032D0001092A9011092A80142C08D518093AA01B9
:1032E000833099F038F4813069F08230D9F48AE67D
:1032F00090E00DC0853099F078F0863099F484E63E
:1033000090E005C08BE690E002C089E690E09093E3
:10331000A9018093A80123C088E690E0F8CF85E654
:1033200090E0F5CF1092AA011AC080E0089586EFD0
:10333000E091A801F091A901309789F02081082E31
:10334000000C990B820F911D8F3F910519F014F01D
:103350008FEF04C097FF02C0108201C0808381E01C
:1033600008950F931F9341E050E060E070E08A0100
:103370009B0104C0000F111F221F331F8A95D2F733
:10338000C901B8010E9463081F910F910C940B08AA
:103390008B3109F468C058F58B3009F486C078F495
:1033A000863009F445C020F4853009F44BC07FC055
:1033B000873009F44AC0883009F477C078C080317A
:1033C00009F464C068F48E3009F071C080919701EF
:1033D00082FB222720F991E0922790FB82F94CC0D2
:1033E000863109F462C0893109F45FC060C08A3255
:1033F000E1F060F4873209F455C028F48E3108F406
:1034000056C08D5150C08932E9F051C0833450F418
:103410008A3308F045C0853309F444C0883309F481
:1034200044C045C08334F1F142C00E94EF0E3DC05C
:1034300080919701817F8E7F8093970181E08093B7
:10344000AB0108950E94C40330C080919701982F6A
:103450009095917090FB80F980939701911125C010
:10346000897F877F10C08091970181FB222720F9F7
:1034700091E0922790FB81F9809397019923A9F01D
:10348000809197018160809397010FC0809197018F
:1034900083FB222720F991E0922790FB83F9ECCF60
:1034A000895301C080E00E94B11981E0089580E055
:1034B000089580E008950C94591ACF93C82F8091F5
:1034C000AB01813069F038F08230C1F58C2F0E9459
:1034D0002F1981E039C00E945E0D823289F504C047
:1034E0000E945E0D823261F48C2F0E945B1A811162
:1034F00004C08C2F0E94C8191FC081E090E01CC03E
:103500008C2F0E94591A811116C0C43189F058F4C9
:10351000CB3089F0C031B1F482E08093AB0188E315
:103520000E942F1908C0C93219F0C83321F00AC00F
:103530001092AB0107C081E0817006C01092AB0110
:1035400080E002C080E0F8CFCF910895CF93DF9361
:1035500086319C4541F5EB010E945E0D982F8A81D2
:103560002091620030916300882379F09A7A81E09B
:1035700009F480E08093AC01911102C069E201C0BE
:1035800065E3C9010E94391C0AC08091AC01811118
:1035900002C069E201C065E3C9010E943B1C0E94B0
:1035A000A00D80E001C081E0DF91CF9108950F93DD
:1035B0001F93CF93DF93C42FD22FFC0182818823E6
:1035C000C9F04093AF010E94761C9093AE018093A6
:1035D000AD0180E28C0F883008F057C0C77081E0E1
:1035E00001C0880FCA95EAF7DF91CF911F910F9123
:1035F0000C9468058091AF01481330C08091AD01F3
:103600009091AE010E948E1C883C910538F510E225
:103610001D0FCD17B9F080E28C0F883040F4C770D1
:1036200081E001C0880FCA95EAF70E946F05183043
:1036300028F581E09D2F977001C0880F9A95EAF7D1
:103640000E946805802F0E945F051830F0F4D77043
:1036500081E001C0880FDA95EAF70AC080E28C0F9A
:10366000883098F4C77081E001C0880FCA95EAF7E6
:10367000DF91CF911F910F910C946F05802FDF91F7
:10368000CF911F910F910C945F05DF91CF911F9106
:103690000F9108950F939C01CB01243F4CE5340713
:1036A00031F188F4293DFCE53F07D9F02A3D4CE58E
:1036B000340779F1283D3C45A9F506E221EE41EEBB
:1036C00068ED7CE52BC0263FFCE53F07E1F0A8F064
:1036D000273F3C4539F507E225EE46EE67EF7CE5EE
:1036E0001DC007E225EE45EE69ED7CE517C006E258
:1036F00021EE40EE64EF7CE511C007E225EE44EEDA
:1037000065EF7CE50BC006E221EE42EE66EF7CE55C
:1037100005C008E221E045EE6AED7CE50E94D71A7B
:1037200080E008C0FC018281882319F01092AF016B
:1037300001C081E00F9108959093F1008093F00013
:1037400008959093B5018093B4010895E091B40178
:10375000F091B501309721F00190F081E02D0994AE
:1037600080E00895E091B401F091B501309721F027
:103770000280F381E02D09940895E091B401F09165
:10378000B501309739F022E0DC012C930480F581FB
:10379000E02D099408952091B2013091B3012817CA
:1037A000390771F09093B3018093B201E091B401B5
:1037B000F091B501309721F00680F781E02D099452
:1037C00008952091B0013091B1012817390771F0A7
:1037D0009093B1018093B001E091B401F091B501F3
:1037E000309721F00084F185E02D09940895FC01C3
:1037F000329697E080E0915029F021912223D9F36D
:103800008F5FF9CF0895662349F0FC013296089640
:103810002191621729F0E817F907D1F780E00895A0
:1038200081E008959C01FC0132969FEF80E0419178
:10383000461789F09F3F19F4411101C0982F8F5FFF
:103840008630A9F79F3F39F0F901E90FF11D97FD87
:10385000FA956283089508959C012A5F3F4FFC0109
:103860004281461301C01282019682179307B9F76D
:1038700008950C94121C0C942C1C029626E0FC015A
:1038800011922A95E9F7089508950C94441C0C941C
:10389000451C0C94441C0C94441C0C94441CCF9365
:1038A0000E944B1C0E94F7120E94491CC0E08C2F02
:1038B0000E942112892B29F4CF5FC830C1F780E024
:1038C00001C081E0CF91089508958091B8018111E0
:1038D0000C942C0408950E940B080C9433048BE084
:1038E00083BF8BEB8CBF82E089BF08952FB7F8941C
:1038F0008091710290917202A0917302B091740252
:103900002FBF08952FB7F8946091710270917202E1
:1039100080917302909174022FBF08959C014FB75C
:10392000F8948091710290917202A0917302B0910B
:1039300074024FBF821B930B089578941F920F92CD
:103940000FB60F9211248F939F93AF93BF938091E3
:10395000710290917202A0917302B091740201966B
:10396000A11DB11D8093710290937202A093730206
:10397000B0937402BF91AF919F918F910F900FBE42
:103980000F901F90189560E081E090E00E948D20DC
:103990009CE088E10FB6F894A89581BD0FBE91BD5B
:1039A000FFCF0E94761C9093B7018093B6010895D3
:1039B0000E94BA1F8B9A80E0815041F0A895E7EBF6
:1039C000FBE03197F1F700C00000F6CF8B987894B8
:1039D00008950E94DD1D0E94A11B2FEB84ED91E054
:1039E000215080409040E1F700C000000895809190
:1039F0009C02882389F010929C020E94761C90936E
:103A0000B7018093B6018091B8018823D1F110925B
:103A1000B8010E946B1C11C08091B801811111C0C6
:103A20008091B6019091B7010E948E1C069728F0F4
:103A300081E08093B8010E94651C8091B8018823C1
:103A400001F10E94651C0E944F1C882339F1F894F3
:103A500021B3939A822F8C6081BB92B38CE098271C
:103A600092BB3FE54AEE90E0315040409040E1F794
:103A700000C0000092B3892782BB21BB9398789441
:103A800008950E94C31E8091A202882329F080918C
:103A9000800284FD0E94DA0F0C94841D08958091A9
:103AA0004D02089508959091BE01981307C020918A
:103AB000BC013091BD0126173707A9F08093BE01E4
:103AC0007093BD016093BC018093B9017093BB01F9
:103AD0006093BA018091B90284FF05C063E089EB6D
:103AE00091E00C94BF1E0895BC0184E00C94531D1A
:103AF000BC0183E00C94531D2091B90224FF03C044
:103B000066E00C94BF1E0895CF93DF93CAE0D0E027
:103B10008091800284FF18C08091CA019091CB01EE
:103B20009817E1F028E0829FC001112468E08453D7
:103B30009E4F0E94BB1E8091CA0190E001968F703B
:103B400099278093CA010AC00E94C31E87EB9BE09D
:103B50000197F1F700C000002197D1F6DF91CF91D6
:103B60000895CF93DF93EC01A091CB01B0E0CD019C
:103B700001968F7099272091CA01281779F093E058
:103B8000AA0FBB1F9A95E1F7A453BE4F98E0FE0120
:103B900001900D929A95E1F78093CB010E94C31E8C
:103BA0000E94841D88E0FE01A2ECB1E001900D921C
:103BB0008A95E1F7DF91CF9108958CE690E0089522
:103BC000FC01808180768032A1F58181813061F4B1
:103BD00084819581892B69F582EC91E090939E0216
:103BE00080939D0288E00895823041F48CE492E055
:103BF00090939E0280939D0281E008958A3021F483
:103C0000838180934C0215C0893099F4828193811D
:103C10008115924081F484819581892B61F481E042
:103C20008093C101868197819093C0018093BF01E9
:103C300002C080E008958FEF08952091BF01309178
:103C4000C001232B71F02091C101213051F4FC01FE
:103C5000808180934D021092C0011092BF0181E0DB
:103C600008958FEF08950895FC0193819330D9F062
:103C700068F4913081F0923009F059C08CE792E0FD
:103C800090939E0280939D028BE30895913249F1B7
:103C90009232B9F14CC087EB92E090939E028093F0
:103CA0009D0282E108958281813099F050F0823046
:103CB000F1F589EC92E090939E0280939D028EE054
:103CC000089587EF92E090939E0280939D0284E096
:103CD000089589ED92E090939E0280939D028CE17D
:103CE00008958281882329F0813009F587EA92E0DE
:103CF00002C08EE892E090939E0280939D0289E03C
:103D0000089584819581009751F0019781F48BEF9C
:103D100092E090939E0280939D028BE7089586E740
:103D200093E090939E0280939D0280E4089580E04A
:103D300008951F93CF93DF93162FEA01288124FF64
:103D400005C0398128E82327298302C02AE5288372
:103D5000212FFC01CE010296DC0131913D932150CF
:103D60001216DCF3612F0E940F021C5F1883DF9193
:103D7000CF911F91089540E852E00C94991E49EBB1
:103D800052E00C94991ECF93DF9360919F02635091
:103D900067FD93C080919B02CCE0D0E0C81BD109A5
:103DA000CD55DD4F80919A02803120F4CE010E94E2
:103DB000331E81C08D3209F06EC0683009F07BC0BF
:103DC00083EC809375028AE58093790010929902C2
:103DD0008881807621F0CE010E94E01D49C09A8141
:103DE00010927E028981811106C010927F022EE717
:103DF00032E082E038C0853019F49093A00230C0E0
:103E00008630A1F48B81813041F0823031F08330F3
:103E100021F0813211F0823221F4CE010E94341E51
:103E200001C080E090E49093990222C0883089F02C
:103E3000893019F49093A20213C08A3069F08B3054
:103E400079F48BE4809381028093BA0280938D028F
:103E500007C022EA32E002C02EE732E081E003C070
:103E60002EE732E080E030939E0220939D0209C04D
:103E70008F3F39F4988197FD8E8190E89093990255
:103E800007C09F81911104C09E81981708F4892F63
:103E90008093780010C08091990287FF0CC0CE01FA
:103EA0000E941D1E8F3F21F48EE18093790003C094
:103EB00081111092780010929F028091790084FF06
:103EC0004CC0809178008F3F09F447C0C82F8930DB
:103ED00008F0C8E08C1B809378009091750288E808
:103EE000892780937502CC2359F180919D0290918E
:103EF0009E022091990226FF12C0A5E7B2E02C2F66
:103F0000AC0145575240FA01EA0FFB1FE4911196AC
:103F1000EC931197215011962111F5CF08C0E6E7D7
:103F2000F2E0DC012C2F3D9131932150E1F7019615
:103F30002FEF2C0F820F911D90939E0280939D0274
:103F40006C2F86E792E00E940F02CC5FCC3019F014
:103F50008FEF80937800C093790084E190B39C70D8
:103F600031F48150D9F71092A00210929802DF919B
:103F7000CF910895CF93DF9385B7886085BF8BB7C6
:103F800080688BBFC0E8D2E08BE48983A9EBB2E004
:103F900011968C931197ECE8F2E081838AE588838F
:103FA0008C938083DF91CF910895DB018F939F9352
:103FB0000E944420BF91AF91A29F800D911DA39FAD
:103FC000900DB29F900D11240895AA1BBB1B51E1C7
:103FD00007C0AA1FBB1FA617B70710F0A61BB70B79
:103FE000881F991F5A95A9F780959095BC01CD011E
:103FF000089597FB072E16F4009407D077FD09D09B
:104000000E94E51F07FC05D03EF4909581959F4FD7
:104010000895709561957F4F0895A1E21A2EAA1B0D
:10402000BB1BFD010DC0AA1FBB1FEE1FFF1FA21768
:10403000B307E407F50720F0A21BB30BE40BF50B65
:10404000661F771F881F991F1A9469F760957095EE
:10405000809590959B01AC01BD01CF010895EE0FB5
:10406000FF1F0590F491E02D0994A29FB001B39F2A
:10407000C001A39F700D811D1124911DB29F700D71
:10408000811D1124911D08950E943520A59F900D3A
:10409000B49F900DA49F800D911D11240895FB01E4
:1040A000DC0104C08D910190801921F441505040F1
:1040B000C8F7881B990B0895E199FECF9FBB8EBB73
:1040C000E09A99278DB30895A8E1B0E042E050E06E
:1040D0000C949C20262FE199FECF9FBB8EBBE09ACB
:1040E00001970DB2021631F02DBB0FB6F894E29A8B
:1040F000E19A0FBE08950396272F0E946B200E941D
:104100006A20252F0E946B20242F0C946B2001968F
:10411000272F0E946B200C946A20262FE199FECF56
:104120009FBB8EBB2DBB0FB6F894E29AE19A0FBEEF
:1041300001960895DC01CB01FC01E199FECF06C098
:10414000FFBBEEBBE09A31960DB20D92415050404C
:08415000B8F70895F894FFCFC1
:10415800C8007501280850011E0A14014F1DB11D21
:104168007C1D781D741D521DFF5AE200E900EA000B
:10417800B500B600B700CD008301CC008A019201DA
:1041880094012102230224022502260227022A0280
:10419800B300B4006F007000818283E200E900EA96
:1041A80000B500B600B700CD008301CC008A0192AB
:1041B8000194012102230224022502260227022A51
:1041C80002B300B4006F00700081828390919293D3
:1041D80094959697373635606162636465666700C3
:00000001FF
